:100000000C9450020C9478020C9478020C947802B0
:100010000C9478020C9478020C9478020C94780278
:100020000C9478020C9478020C9403240C94D2243F
:100030000C94311F0C9478020C9478020C94780282
:100040000C9478020C9478020C9478020C94780248
:100050000C9478020C948E1F0C9478020C94780205
:100060000C9478020C9478020C9478020C94780228
:100070000C9478020C9478020C9478020C94780218
:100080000C9478020C9478020C9478020C94780208
:100090000C9478020C9478020C9478020C947802F8
:1000A0000C9478020C9478020C947802350535058E
:1000B00061056105C905E705FF06FF06F2058B0628
:1000C0009C069C063F2566255E2666255E26B22593
:1000D000D5255E262C263B262B0014001A0008008E
:1000E000150017001C0018000C00120013002A0055
:1000F000296104001600070009000A000B000D002A
:100100000E000F0033002861E1001D641B00060093
:1001100019000500110010003600370038644C62E9
:100120000000000000002F412C43346831682C424D
:10013000304100000000000035001E001F002000BC
:1001400021002200230024002500260027002E0085
:1001500049001E021F022002210222022302240261
:100160002502260227022D003A003B003C003D00FC
:100170003E003F0040004100420043004400450073
:100180000000000000003900DE5C2A5D0100010073
:1001900001000000000000000100010001004B0010
:1001A00001000100BD00010052000100010001003A
:1001B000010001004A004E004D0001000100500006
:1001C00051004F0001000100010001000100010089
:1001D00001000100BE00AA00A800A9000100010062
:1001E000000000000000010001000100010001000A
:1001F000010000000000000001000100B900F9004A
:10020000B40001000100F100ED00F2000100010066
:1002100001000100FB00FA00FC0001000100EF00FA
:10022000EE00F0000100010001000100AC00AE0092
:10023000AB0001000100010001000100010001000C
:1002400000000000000001000100010001000100A9
:10025000010000000000000041542B424C45484979
:10026000444D4F555345425554544F4E3D00415413
:100270002B424C454849444D4F5553454D4F5645EB
:100280003D25642C25642C25642C25640041542BC9
:10029000424C45484944434F4E54524F4C4B4559AC
:1002A0003D3078253034780041542B424C454B4545
:1002B00059424F415244434F44453D253032782DF9
:1002C00030302D253032782D253032782D253032C2
:1002D000782D253032782D253032782D2530327822
:1002E0000041542B474150474554434F4E4E004127
:1002F000542B4556454E54454E41424C453D307871
:10030000320041542B4556454E54454E41424C45D2
:100310003D307831004F4B004154453D3000415451
:100320002B4741504445564E414D453D34320041E6
:10033000542B424C45484944454E3D310041542BD5
:10034000474150494E54455256414C533D31302C53
:1003500033302C2C0041545A0041542B424C455010
:100360004F5745524C4556454C3D2D3132001803F0
:100370003D031E032F0359035503060334003200C7
:1003800000000E036E0067006C0067007A007A00C0
:1003900000000403090409023B00020100A0FA095D
:1003A00004000001030101000921110100012240A4
:1003B0000007058103080001090401000103000092
:1003C00000092111010001227B00070582032000A2
:1003D000011201000200000008EDFE000003000110
:1003E00002000105010902A10185020901A1000520
:1003F00009190129081500250195087501810205D3
:1004000001093009311581257F950275088106099A
:10041000381581257F950175088106050C0A38027B
:100420001581257F950175088106C0C005010980E9
:10043000A101850319012AB700150126B70095010E
:1004400075108100C0050C0901A101850419012A5C
:10045000A002150126A002950175108100C00501BA
:100460000906A101050719E029E7150025019508EE
:10047000750181029501750881010507190029FFA1
:10048000150026FF00950675088100050819012949
:1004900005950575019102950175039101C0631CD5
:1004A00011241FBECFEFDAE0DEBFCDBF11E0A0E028
:1004B000B1E0ECEEF4E502C005900D92AA3AB10766
:1004C000D9F724E0AAEAB1E001C01D92A432B20734
:1004D000E1F712E0C0E5D2E004C02197FE010E94DE
:1004E000AC26CF34D107C9F70E94EA120C94742AC3
:1004F0000C94000081E0089581E008950C947C0242
:1005000008950C9480021F93CF93DF9300D000D006
:100510001F92CDB7DEB749835A836B833091AD010B
:1005200089819A81311114C0662359F0222349F040
:100530000E943C09182F682F89819A810E94E50842
:1005400003C00E941009182F69817A81812F04C08D
:100550000E943C0969817A810F900F900F900F9053
:100560000F90DF91CF911F910C946C10FC01262FFE
:10057000408151816281738184810C94830281E086
:100580000895CF93DF93EC0160E00E94B602BE01B4
:10059000DF91CF910C9481020C949B110C949711D4
:1005A00008950E948F070E94D0022FE78AE196E00B
:1005B000215080409040E1F700C000000C94B41F2F
:1005C0000F931F93CF93DF938C0161E00E94B602DB
:1005D000EC01B8010E947E02882309F451C0B801E1
:1005E000CE010E94101D882309F44AC0B801CE0133
:1005F0000E948015882309F443C0B801CE010E94EF
:100600006C1C8823E9F1F8018281882391F1CF3DA8
:100610008CE5D80701F158F4CD3DFCE5DF07F1F09A
:10062000F8F4C115DC4529F50E94D10229C0CB356B
:10063000FDE5DF07C9F028F4CA32DD45D1F483E0D7
:1006400010C0CC35FDE5DF0791F0CD35DD4589F4EF
:100650000E94B60D0EC00E946D0E12C080E001C057
:1006600082E00E94C9160CC00E94BF0D02C00E9409
:10067000C20DC801DF91CF911F910F910C947A02A6
:1006800080E0DF91CF911F910F9108950E945B034D
:100690000C942E1F08950C944A0381E008950C9445
:1006A0004D030895CF93C82F0E944B038C2F0E94B7
:1006B0004F03CF9108950E94751E0C9452030E941F
:1006C000751E9091AC01891721F08093AC010C94B8
:1006D00052030895CF93DF93CDB7DEB72B970FB6B4
:1006E000F894DEBF0FBECDBF4F83588769877A87E6
:1006F0008B8761110E94020D9E012F5F3F4F86E0A4
:10070000F90111928A95E9F785E0FE013796D90142
:1007100001900D928A95E1F789819A814C815D81E2
:10072000452B31F09F3F31F491E08F3F19F403C026
:1007300091E001C090E090FF09C049815A816B812E
:100740007C818D819E810E94230C05C0C9010E947D
:10075000BF028111F2CF2B960FB6F894DEBF0FBE09
:10076000CDBFDF91CF910895FC01808191810E94DE
:100770007E090895CF93882309F4A4C0C82F823836
:10078000C1F40E94751E81FD9DC069E38091020144
:10079000909103010E94081F0E94240D2FEF80E713
:1007A00092E0215080409040E1F700C0000069E3F2
:1007B00019C0833801F50E94751E80FD83C063E572
:1007C00080910201909103010E94081F0E94240D54
:1007D0002FEF80E792E0215080409040E1F700C089
:1007E000000063E580910201909103010E940A1FBD
:1007F000CF910C94240D8438C1F40E94751E82FDA3
:1008000061C067E480910201909103010E94081F7A
:100810000E94240D2FEF80E792E02150804090400D
:10082000E1F700C0000067E4DDCF8CEF8C0F813A68
:10083000D0F46C2F80910201909103010E94D21E8E
:10084000882349F06C2F80910201909103010E944E
:100850000A1F0E94240D6C2F8091020190910301C8
:100860000E94081FC5CF80E28C0F883048F4C77003
:1008700081E001C0880FCA95EAF70E94E50CB8CF65
:10088000EBE5EC0FE33040F4F0E0E75BFE4F8081F6
:1008900090E0CF910C949A1EE8E5EC0FE73150F40C
:1008A000F0E0EE0FFF1FE55EFE4F80819181CF915A
:1008B0000C94B01ECD3E30F08C2F0E946F13CF9160
:1008C0000C944114CF910895882309F464C08238B0
:1008D00079F40E94751E81FF5EC069E38091020178
:1008E000909103010E94081F0E94240D69E310C02B
:1008F0008338B1F40E94751E80FF4DC063E580917E
:100900000201909103010E94081F0E94240D63E5DB
:1009100080910201909103010E940A1F0C94240D02
:10092000843879F40E94751E82FF35C067E4809197
:100930000201909103010E94081F0E94240D67E4A8
:10094000E7CF9CEF980F913A10F4682FE1CF90E237
:10095000980F983050F4877091E001C0990F8A95F4
:10096000EAF7892F0E94EB0CD9CF9BE5980F9330C3
:1009700020F480E090E00C949A1E98E5980F97314F
:1009800020F480E090E00C94B01E8D3E20F00E9498
:10099000CA130C94411408951F93CF93DF93182F1B
:1009A000EB010E94BA03209741F08FEC97E001978A
:1009B000F1F700C000002197F6CF812FDF91CF9192
:1009C0001F910C946404893319F060E070E002C058
:1009D00060E570E00C94CC04882321F00E94E50CC3
:1009E0000C94240D0895882321F00E94EB0C0C94A4
:1009F000240D0895CF92DF92EF92FF920F931F93F1
:100A0000CF93DF937C01D62FC72FFC011281058184
:100A100002950F700E94DB0C8823B9F01123A9F016
:100A20008C2F807F803421F080E28D0F883068F039
:100A30008091020482FD09C082E00E94840D0E9420
:100A4000DB0C91E0D82ED92601C0D12CCC2EC2943B
:100A50008FE0C8228C2D90E08C30910508F0CFC13A
:100A6000FC01EA5AFF4F0C94AC268C2F807FCF708C
:100A7000882311F0C295C07F112399F0CC2309F48B
:100A8000AAC180E28D0F883010F0D11104C08C2FE4
:100A90000E94E50C03C08C2F0E94F50C0E94240DCF
:100AA0009AC18D2F0E946404CC2309F4A8C180E26E
:100AB0008D0F883038F1DD2329F18C2F0E94FB0C3B
:100AC00024C08C2F807FCF70803211F0C295C07F00
:100AD000DD2319F0D130A1F13DC08091020482FFE5
:100AE00017C0112349F0CC2329F08C2F0E94E50C6C
:100AF0000E94240D80E070C180E00E946404CC2339
:100B000009F47DC18C2F0E94EB0C0E94240D77C14B
:100B1000112371F0002341F0013031F40E94050DE2
:100B20008C2B0E940D0D6BC10E94050D8C2B1DC0DE
:100B3000002319F0013009F462C10E941A0D25C08A
:100B4000112321F0063008F05AC10EC0053008F01C
:100B500056C11BC0112361F0002331F0F7018581DC
:100B600080FF39C18F7085838C2F0E94EC0447C1B0
:100B7000002359F0D93309F03FC1FFEF03EF11E033
:100B8000F15000401040E1F735C18C2F0E94F30472
:100B900036C18C2F86958695837019F0813061F06F
:100BA0002EC1112321F08D2F9C2F937002C080E065
:100BB00090E00E949A1E2BC1112321F08D2F9C2FB3
:100BC000937002C080E090E00E94B01E20C18D2F83
:100BD000112319F00E946F1302C00E94CA130E94D1
:100BE000411415C18C2F837009F047C011110BC13E
:100BF0002D2F229526952770220F220F6D2F6F70B3
:100C0000862F90E0A0E0B0E0022E04C0880F991F6C
:100C1000AA1FBB1F0A94D2F7D4FF10C04FE050E0C8
:100C200060E070E004C0440F551F661F771F2A95CF
:100C3000D2F7409550956095709503C040E050E024
:100C4000BA01C695C695C3708A019B01082B192B62
:100C50002A2B3B2BC901B801C23049F058F4C130EE
:100C600019F00E94FB07CFC00E94E907CCC00E9488
:100C70000D08C9C00E94E707C6C0112319F08C2FC8
:100C8000817001C08695882309F4BDC02D2F22955F
:100C900026952770220F220F6D2F6F70862F90E000
:100CA000A0E0B0E0022E04C0880F991FAA1FBB1F4E
:100CB0000A94D2F7D4FF10C04FE050E060E070E03B
:100CC00004C0440F551F661F771F2A95D2F7409521
:100CD00050956095709503C040E050E0BA01C6950C
:100CE000C695C3708A019B01082B192B2A2B3B2B1D
:100CF000C901B801C23049F058F4C13019F00E945E
:100D0000C00881C00E94AE087EC00E94D2087BC08D
:100D10000E94210878C0CF70112339F08C2F0E94D7
:100D200047088D2F0E94EC046EC08D2F0E94F304A3
:100D30008C2F0E94680867C0D23F21F128F4D03F71
:100D400041F0D13FC1F043C0D33F19F1D43F79F016
:100D50003EC0112341F0053008F051C08C2F8F7137
:100D60000E948D084CC0063008F049C0F7CF809132
:100D7000020482FF18C0112339F08C2F8F710E945A
:100D800047083DC01123C9F38C2F8F710E9468085A
:100D900036C0112329F08C2F8F710E9432082FC08A
:100DA0000E942D082CC0112349F0CF718C2F0E9476
:100DB000470863E08C2F0E94690D21C081E00E94EA
:100DC000840D0230E0F082E00E94840D18C01123EF
:100DD00031F0002391F28D2F0E94BA0310C000233E
:100DE00099F2D93349F41FEF23EF31E0115020403D
:100DF0003040E1F700C000008D2F0E94640488EFAE
:100E00008C0D843020F40E94751E0E945203DD2058
:100E1000C9F00E94D70C80FD15C0F70112820E9414
:100E2000D10C0E944708C7010E9443070E94D10CC1
:100E3000DF91CF911F910F91FF90EF90DF90CF90B6
:100E40000C946808DF91CF911F910F91FF90EF9064
:100E5000DF90CF9008950F931F93CF93DF93EC0112
:100E6000688179818A810E9489098C010E94E40845
:100E70000E94D507B801CE010E94FA04DF91CF91FC
:100E80001F910F910895CF93DF93EC019881898191
:100E90002B813C81232B31F08F3F31F481E09F3F48
:100EA00019F403C081E001C080E080FD1DC0CE01C7
:100EB0000E94E002811110C00E94DB0C8823A1F087
:100EC0008A81882389F08091020482FD0DC082E02E
:100ED000DF91CF910C94840DCE010E942B07CE019F
:100EE000DF91CF910C94C102DF91CF91089580E002
:100EF00090E00E949A1E80E090E00E94B01E0E9446
:100F0000020D0E94240D0E9472150C9441148091D0
:100F10000201909103010E940C1F0C9477070E941C
:100F2000F20C0C94870792959F70963079F010F42C
:100F3000925001C09A50923068F4803F69F018F4E2
:100F4000883E40F409C0843F29F406C0883E20F062
:100F5000813F11F080E0089581E00895FC018081D7
:100F600091810E947E090E9493070895CF93DF9399
:100F700000D000D01F92CDB7DEB70F900F900F902A
:100F80000F900F90DF91CF910895CF93DF9300D012
:100F900000D000D0CDB7DEB726960FB6F894DEBFEE
:100FA0000FBECDBFDF91CF910895089508950C94A1
:100FB000D6070C94D7070E94D9076093D00170938D
:100FC000D1018093D2019093D3010C9477070C94B4
:100FD000DB070F931F930091D0011091D101209155
:100FE000D2013091D301602B712B822B932B1F9157
:100FF0000F910C94DB070F931F930091D001109178
:10100000D1012091D2013091D30160237123822339
:1010100093231F910F910C94DB070F931F93009163
:10102000D0011091D1012091D2013091D3016027DC
:101030007127822793271F910F910C94DB070C9443
:10104000D6070E941F086093CC017093CD01809356
:10105000CE019093CF010C94770760E070E0CB0154
:101060000C9421080F931F9341E050E060E070E082
:101070008A019B0104C0000F111F221F331F8A9594
:10108000D2F7C901B8011F910F910C9421080F9359
:101090001F9341E050E060E070E004C0440F551F32
:1010A000661F771F8A95D2F78091CC019091CD0170
:1010B000A091CE01B091CF018A019B01082B192B81
:1010C0002A2B3B2BC901B8011F910F910C942108C9
:1010D0000F931F9341E050E060E070E004C0440FC4
:1010E000551F661F771F8A95D2F7409550956095DA
:1010F00070958091CC019091CD01A091CE01B091DD
:10110000CF018A019B01082319232A233B23C9010C
:10111000B8011F910F910C9421080F931F9341E088
:1011200050E060E070E004C0440F551F661F771F59
:101130008A95D2F78091CC019091CD01A091CE01FA
:10114000B091CF018A019B01082719272A273B2745
:10115000C901B8011F910F910C9421080F931F939F
:101160000091CC011091CD012091CE013091CF01A1
:10117000602B712B822B932B1F910F910C942108C4
:101180000F931F930091CC011091CD012091CE01BE
:101190003091CF0160237123822393231F910F91FC
:1011A0000C9421080F931F930091CC011091CD0155
:1011B0002091CE013091CF0160277127822793279C
:1011C0001F910F910C94210808952CE0929F800D9F
:1011D0001124E82FE695E695E695877051E001C069
:1011E000550F8A95EAF785E0E89FF0011124E25552
:1011F000FE4F20E030E070E04081CB01022E02C0C3
:10120000969587950A94E2F78170819584278523C6
:10121000842781932F5F3F4F2530310569F708956B
:101220002CE0929F800D1124682F66956695669537
:10123000982F977085E0689FB001112440E050E03E
:1012400080E0FB01E40FF51FE255FE4F208130E006
:10125000092E02C0369527950A94E2F721703327AC
:10126000042E01C0220F0A94EAF7822B4F5F5F4FD2
:101270004530510531F70895BF92CF92DF92EF923A
:10128000FF920F931F93CF93DF938C01C090CC01FB
:10129000D090CD01E090CE01F090CF018091D001AF
:1012A0009091D101A091D201B091D301C82AD92A3D
:1012B000EA2AFB2ACFE1D0E0D701C6010C2E04C0F8
:1012C000B695A795979587950A94D2F780FD04C0A7
:1012D000219790F7B12C07C0BC2EB8018C2F0E942B
:1012E0007F100197A9F38B2DDF91CF911F910F9163
:1012F000FF90EF90DF90CF90BF900895CF93DF9352
:10130000EC010E943C09BE010E947F10DF91CF9149
:1013100008951F93CF93DF93EB019091AD01992333
:1013200021F0CB010E947E0913C0882349F0CB0134
:101330000E943C09182F682FCE010E94E50804C0C6
:10134000CB010E941009182FBE01812F0E947F102F
:10135000DF91CF911F9108951F93CF93DF93C09199
:10136000D40116E08091D501C81799F0D0E01C9FF8
:10137000F0011D9FF00D1124EA52FE4F4081518172
:1013800062817381848195810E94C5072196C7700F
:10139000E9CFDF91CF911F910895409106025091BE
:1013A0000702609108027091090280910A029091EF
:1013B0000B020C94C507EF92FF920F931F93CF93EC
:1013C000DF9380910B0282958F7009F065C0809148
:1013D0000802882309F460C08091D401F090D501FF
:1013E00010910602009107026091090270910A02B1
:1013F00091E01F3F09F090E0C0910001D091010100
:10140000292F96E0E92E8F1509F446C06115710564
:1014100021F00F3F21F030E003C031E001C0322F56
:1014200090E030FD36C0E89EF001E99EF00D1124F9
:10143000DF01AA52BE4F11963C911197301329C07B
:101440003C91311326C012963C911297311121C064
:1014500013964D915C911497461B570B4C175D07E3
:10146000C0F480910B028F70806180930B02E55273
:10147000FE4F80818F708061808386E092E00E94C1
:101480004307DF91CF911F910F91FF90EF900C9444
:10149000AC0901968770B7CFDF91CF911F910F9163
:1014A000FF90EF9008959F92AF92BF92CF92DF92FC
:1014B000EF92FF920F931F93CF93DF93CDB7DEB7D9
:1014C00061970FB6F894DEBF0FBECDBF8C0185E0EB
:1014D000F801DE011D9601900D928A95E1F7D80181
:1014E0001296EC9090910602E09107022091090279
:1014F00030910A022115310531F0EF3F31F481E0DE
:101500009F3F19F403C081E001C080E0B82FB170A3
:101510009B2E80FD47C1D8014C9111965C9111978B
:101520001396AD90BC90149786E0C82E82E0D82E1A
:10153000F0900802B501621B730B209100013091FD
:101540000101FF2009F4D9C080910B0262177307D3
:1015500008F095C0282F207F09F052C05E1313C0F9
:10156000491311C0FE2CE1100EC08F708061809372
:101570000B020E94CD09C6010E94430780910B0215
:10158000F80185834DC1AB2831F05F3F31F481E034
:101590004F3F19F403C081E001C080E080FD03C02B
:1015A00081E08E2502C080E090E0F82FF170FF2EE0
:1015B00080FF1CC08091D4012091D50136E08217B4
:1015C00009F40BC190E0389FF001399FF00D112410
:1015D000EA52FE4F6181561306C06081461303C074
:1015E0006281E61203C001968770E9CFFE2CEE20DF
:1015F00009F416C180910B02816080930B0254C0E4
:101600005E1306C0491304C0E11002C0F80199C07E
:10161000C8010E94AE07882361F1EE2051F12091AC
:101620000B02822F82958F7090E0029774F0809168
:1016300006029091070298878F831986BB86AA8637
:101640002C87CE0107960E94430786E0F801A6E0AA
:10165000B2E001900D928A95E1F70E94DB090E94A9
:10166000CD090AC05E1711F1C8010E94AE078111B1
:101670002CC0C8010E944307FF24F394D1C0282F37
:10168000207F81F77A2DB98AA88A6E2D89890E94D8
:10169000B60786E092E00E94430786E0D6011D92DD
:1016A0008A95E9F70E94CD09F12CBAC04913DCCF25
:1016B000E110DACFF8018583C8010E94430786E074
:1016C000D6011D928A95E9F7ABC0EE2091F22091E8
:1016D0000B02822F82958F7090E002970CF4B5CFA9
:1016E00080910602909107029A8389831B82BD82B2
:1016F000AC822E83CE010196A6CF6217730708F045
:1017000044C0FE2CEE2009F4B4CF5E1330C0491360
:101710002EC020910B0220FD21C0822F82958F7058
:10172000482F50E041155105C9F0F80125834F308D
:10173000510541F08F5F982F9295907F822F8F7087
:10174000892B8583C8010E94430786E0F801A6E043
:10175000B2E001900D928A95E1F73CC086E0F80175
:10176000A6E0B2E001900D928A95E1F759C0C80158
:101770000E94AE07811169CF80910B028160809336
:101780000B02C8010E9443074BC07A2DB98AA88A70
:101790006E2D89890E94B60786E0D6011D928A9532
:1017A000E9F718C0EE2009F464CFC8010E94AE0723
:1017B000F82E882309F45DCF86E0F801A6E0B2E0B8
:1017C00001900D928A95E1F786E092E00E94B403C1
:1017D0000E94DB090E94CD0923C04D875E878D855D
:1017E0009E850E947E09292F22952F70223028F491
:1017F0009F7039F0811105C00BC0243028F49F7010
:1018000049F4805E883020F0C8010E9443079F2C75
:10181000F92C06C0D80115969C91907F91F7F8CFCE
:101820008F2D61960FB6F894DEBF0FBECDBFDF914E
:10183000CF911F910F91FF90EF90DF90CF90BF90CD
:10184000AF909F9008951F93CF93DF93CDB7DEB7EE
:101850002C970FB6F894DEBF0FBECDBF4F835887CD
:1018600069877A878B879C87CE0107960E94530AE7
:101870008823D1F09F8188852A853B85232B31F0F1
:101880008F3F31F481E09F3F19F403C081E001C034
:1018900080E080FD47C04F81588569857A858B85BA
:1018A0009C850E94C5073EC086E0FE013796DE019A
:1018B000119601900D928A95E1F7FF81E8856A857E
:1018C0007B856115710531F0EF3F31F481E0FF3F19
:1018D00019F403C081E001C080E080FD23C02091A5
:1018E000D50130E0C9010196877099274091D40154
:1018F00050E084179507F1F1F983EA837D836C83C7
:1019000096E0929FD001939FB00D1124AA52BE4F32
:10191000FE01319601900D929A95E1F78093D501E1
:101920000E94AC0916E08091D4019091D5018917ED
:1019300071F1189FC00111248A529E4F0E94530AD0
:10194000882329F1E091D4011E9FF0011124EA526D
:10195000FE4F4081518162817381848195810E9413
:10196000C5078091D40190E00196877099278093F4
:10197000D401D9CF0E948F071092D5011092D401C3
:10198000E6E0F2E086E0DF011D928A95E9F72C9609
:101990000FB6F894DEBF0FBECDBFDF91CF911F9180
:1019A0000895809114028595859585950895809177
:1019B00014028770089590911402977081E009F4E1
:1019C00080E0089580911F02089590911F02892B55
:1019D00080931F020895809590911F028923809320
:1019E0001F02089510921F02089590911E02892BE4
:1019F00080931E020895809590911E028923809302
:101A00001E02089510921E020895809115020895F5
:101A100008950C94080D0C94090D9091020492FD08
:101A200008C090911502981721F0809315020C942C
:101A30000B0D089580911502882329F0109215024C
:101A400080E00C940B0D0895CF93DF93E091020199
:101A5000F091030180911F028083E0910201F091D7
:101A60000301908180911E02892B80838091150251
:101A7000882381F0E0910201F09103019081892B8C
:101A8000808380910201909103010E94C61E811102
:101A90000E941A0DC0910201D091030148E050E06C
:101AA0006CE072E0CE010E940627892B69F088E085
:101AB000FE01ACE0B2E001900D928A95E1F7CE0113
:101AC000DF91CF910C94811EDF91CF9108950C94FA
:101AD000080D9091020492FD10C098E0899F90013A
:101AE0001124262B209314020E944708809114028F
:101AF0008595859585950C94670D0C9447081092F3
:101B0000140280E00C94670D2091140280958223CA
:101B100080931402982F977099F430E0482F082E84
:101B2000000C550B2417350759F09091020492FDD3
:101B300007C08595859585950E9468080C947F0D52
:101B400008959091020492FB222720F9281769F04A
:101B500080FB92F990930204809101049091020419
:101B60000E94E90D82E00C94840D08958091020496
:101B700082FB882780F991E089270C94A10D81E0F0
:101B80000C94A10D80E00C94A10D80E090E00E94E7
:101B9000032A21E0893E9E4F09F020E0822F08951C
:101BA00082E090E00C94FB2983E090E00C94FB2908
:101BB000CF9384E090E00E94FB29C82F82E290E05E
:101BC0000E94FB292C2F30E0A901582BCA01CF918C
:101BD0000895CF93C92F682F84E090E00E94092ACE
:101BE0006C2F82E290E0CF910C94092AAB01BC01EA
:101BF0008FE090E00C941B2AAB01BC0183E190E0E4
:101C00000C941B2A60E070E0CB010C94FC0D60E0AA
:101C100070E0CB010E94F60D0C94020E69EE7EEF8F
:101C200080E090E00E94272A60E082E090E00E943D
:101C3000092A60E083E090E00E94092A1092D00116
:101C40001092D1011092D2011092D30160E084E091
:101C500090E00E94092A60E082E290E00E94092A56
:101C600060E085E090E00E94092A60E086E090E074
:101C70000E94092A6FEF87E090E00E94092A40E065
:101C800050E0BA0188E090E00E941B2A60E08DE0FD
:101C900090E00E94092A40E050E0BA0188E190E01B
:101CA0000E941B2A60E087E190E00E94092A40E040
:101CB00050E0BA018CE190E00E941B2A60E070E0E5
:101CC00080E290E00E94272A40E050E0BA0188E1DB
:101CD00090E00E941B2A0C94070E0C940E0E682FA5
:101CE0008EE090E00C94092A0E94731F60932C02EE
:101CF00070932D0280932E0290932F0260932802FE
:101D00007093290280932A0290932B02089585B73D
:101D1000806885BF85B7806885BF089581E0089594
:101D20000C948E0E08950C94920E0C94920E0C94BA
:101D3000950E0C94920E0C94990E0C94920E0E9497
:101D4000870E8BE591E10E946B1E0E949D0E0C9404
:101D50009B0E0E94930E0C94920E0E945E110C94A6
:101D600051030E945E1F0E9443120E94AD0E0C940C
:101D7000970E5F926F927F928F929F92AF92BF92D7
:101D8000CF92DF92EF92FF920F931F93CF93DF9347
:101D9000CDB7DEB72A970FB6F894DEBF0FBECDBF22
:101DA0000E945812C82E81110E94740E30E2832EB8
:101DB00032E0932E00E010E0502E802F0E9482111E
:101DC0005C01F401619071904F01682679266114DD
:101DD0007104B1F40F5F1F4F0430110569F78FEFE5
:101DE00089838A831B820E94671F8160782F9D836D
:101DF0008C8349815A816B818D810E946A033AC02C
:101E00008091300281FD0E948B11D12CEE24E3944D
:101E1000F12CC3018E219F21892B29F10E94900E64
:101E20008823A9F0DE825F82AE20BF2081E0AB284C
:101E300009F480E088870E94671F8160782F9A8765
:101E400089874E815F8168858A850E946A03000FB9
:101E5000111FF801E05EFD4F80819181E826F9268F
:101E6000F182E08207C0D394EE0CFF1CFCE0DF128D
:101E7000D0CFB0CF81E0C11001C080E02A960FB66C
:101E8000F894DEBF0FBECDBFDF91CF911F910F91B0
:101E9000FF90EF90DF90CF90BF90AF909F908F908A
:101EA0007F906F905F9008950E94B90E0E945F141A
:101EB0000C945F03CF93DF930E948410EC01811593
:101EC00021E5920708F045C0811530E5930708F039
:101ED00094C0883E910528F5803E910508F0F8C031
:101EE000883A910570F4853A910508F07CC08130FC
:101EF000910509F475C008F4E8C0049708F0E8C03B
:101F0000E4C08F3B910508F0E0C0C85AD0E0CC0F88
:101F1000DD1FC45BDE4F0990D881C02DCE019464D3
:101F2000D8C0811540E2940758F4811551E0950717
:101F300008F0CEC08D3E910508F4C7C09065C9C0B9
:101F4000C11580E4D80708F4C0C0DF70CE01906AE4
:101F5000C0C0811525E59207A8F4811534E59307E3
:101F600008F095C0811543E5940708F07BC0811502
:101F700052E5950708F061C0D82FCC27CE01816FBC
:101F8000906AA7C0C11589E5D807A0F4C11528E556
:101F9000D20708F082C0C11536E5D30708F095C016
:101FA0008C2F0E9418118F7190E0D82FCC27CE0172
:101FB00090628FC0C1154AE5D40708F474C0CE0101
:101FC00090568115904208F080C08D2F8F710E942D
:101FD0001811DD27D0628F71AE01582BCA0179C06C
:101FE00081E090E076C0C55AD0E0C658DE4F8881C7
:101FF000C82FD0E0CE0190646CC074E096958795B0
:102000007A95E1F7282F23703C2F337081E090E020
:1020100002C0880F991F3A95E2F79C68AC01522BD9
:102020009A019C2F9F709695969550E2959FE0019E
:102030001124C9018C2B9D2B4CC08370992721E062
:1020400030E002C0220F331F8A95E2F79C2F96954D
:10205000969580E2989FE0011124C22BD32BCE01EC
:102060009C6837C08370992721E030E002C0220FBE
:10207000331F8A95E2F79C2F9695969540E2949FA0
:10208000E0011124C22BD32BCE019A6822C0D82F95
:10209000CC27CE01846F906A1CC0DC2FCC27CE01E8
:1020A000806F906A16C08C2F8F700E94181194E078
:1020B000D695C7959A95E1F7CF70D0E0DC2FCC2765
:1020C000D0699E01282BC90104C080E090E001C0C6
:1020D000CE01DF91CF91089520E3829FC0011124AA
:1020E000FC012CE0729FE00DF11D1124E60FF11DA3
:1020F000EE0FFF1FE852FF4F8591949108950E94C3
:102100006C100E945A0F08958238910569F1B0F45D
:102110008133910509F46DC048F48932910509F4C1
:1021200063C08A32910509F469C008958533910529
:1021300009F455C089339105B9F00895833E91059E
:1021400069F138F4803E9105B1F0823E910509F1C4
:102150000895863E9105A9F1873E9105B9F1843E27
:10216000910509F064C023C02091010420FD4FC0F7
:1021700021FD4DC008958091010480FD44C08091EF
:10218000020480FF44C08091010484FD42C083EEBC
:102190004DC08091010482FF38C0F5CF80910104C9
:1021A00082FD33C08091020480FD31C0ECCF80916C
:1021B000020481FF32C08091010484FD2AC087EEB1
:1021C00035C08091010483FF26C0F5CF80910104C2
:1021D00083FD21C08091020481FD1FC0ECCF80915E
:1021E000010485FD1CC01DC08091010485FD19C03E
:1021F00016C08091010486FD16C017C080910104AD
:1022000086FD13C010C089E311C082EE0FC080EEBE
:102210000DC080E00BC086EE09C084EE07C089E2E5
:1022200005C085E303C08AE201C081E390E0089520
:102230009091010492FF0DC0282F2871283019F4C5
:10224000877F846006C0282F2471243011F48B7F8F
:10225000886093FF0DC0282F2871283119F4877EDC
:10226000846106C0282F2471243111F48B7E88618B
:102270002091020420FF0DC0382F3871383019F436
:10228000877F816006C0382F3171313011F48E7F25
:10229000886021FF0DC0282F2871283119F4877E0E
:1022A000816106C0282F2171213111F48E7E886151
:1022B00094FD877E089580E0089508950E94C50DDD
:1022C000811102C00E946D0E0E94D00D80933002D9
:1022D0000E94D80D90930204809301040E945D1126
:1022E0000E94D40D682F70E080E090E00E94E70724
:1022F0006091CC017091CD018091CE019091CF0180
:102300000C941F08E82FF0E0EE0FFF1FE55FFB4F76
:10231000808191810895089580E58A95F1F7089567
:1023200000C008950C948C1108950C9494110C9491
:1023300095110C9494110C949911F894E82FE2954E
:10234000EF70F0E031A1282F2F7081E090E001C004
:10235000880F2A95EAF7982F9095932391A392A13D
:10236000892B82A3789408950F931F93CF93DF93C3
:10237000C9E8D1E089918F3F11F00E949D1181E061
:10238000CD38D807B9F7CDE7D1E009E811E0899158
:102390008F3F11F00E949D110C171D07C1F7DF91AF
:1023A000CF911F910F910895BF92CF92DF92EF923C
:1023B000FF920F931F93CF93DF938C01C62FD0E032
:1023C000CE0187579E4F6C01FC0190819F3F09F41D
:1023D00050C0B62EF894E92FE295EF70F0E081A19D
:1023E0009F7021E030E001C0220F9A95EAF7822B1E
:1023F00081A382A12095282322A378940E94901182
:10240000EDE7F1E049E851E021E030E0E12CF12C8A
:1024100061916F3F89F0A62FA295AF70B0E09096C2
:102420008C9190E06F7002C0959587956A95E2F760
:1024300080FD02C0C90102C080E090E0E82AF92ACC
:10244000220F331F4E175F0719F7F60180818F3F68
:1024500011F00E949D1161E0E114F10409F460E0C3
:102460008B2D0E949211CC0FDD1FC00FD11FF9825E
:10247000E882DF91CF911F910F91FF90EF90DF9055
:10248000CF90BF9008950E94B41188E0EBE0F4E093
:10249000DF01982F1D929A95E9F7E3E0F4E0DF0160
:1024A0001D928A95E9F784E00E94A3120C94CC0255
:1024B000FF920F931F93CF93DF93CDB7DEB728978B
:1024C0000FB6F894DEBF0FBECDBF8E010F5F1F4F5A
:1024D00088E0F80111928A95E9F7F12C6F2DC80177
:1024E0000E94D411F394F4E0FF12F8CF48E050E0DA
:1024F000B80183E094E00E940627FF24F39400973C
:1025000009F4F12C892B41F088E0F801A3E0B4E054
:1025100001900D928A95E1F72F2D44E06BE074E075
:1025200083E094E00E94A4120E94CE028F2D289690
:102530000FB6F894DEBF0FBECDBFDF91CF911F91D4
:102540000F91FF9008950895FF920F931F93CF93DB
:10255000DF93F82E092F162FD72FC42F222349F0EF
:1025600081E0809333020E94671F90933202809330
:102570003102809133028823D9F080913102909109
:1025800032020E947F1F059798F0EF2DF02FA12FA8
:10259000BD2F80E090E04C2F50E08417950734F475
:1025A000219131912D933D930196F7CF10923302F3
:1025B000DF91CF911F910F91FF9008950E94892183
:1025C0000E94B10E0C9495210E9499210E94540FF3
:1025D0000C949A210E94301F0E9470210E949F0E2D
:1025E0000E94DE120E94E4120E94A90EFBCF80918D
:1025F0003A0280FF06C06091090170E0660F771F04
:1026000026C081FF04C06091090184E005C082FFFB
:1026100007C06091090188E0689FB001112417C0CC
:10262000909139029923D1F060910801961788F7AB
:102630002091090188E0289F90011124929FA00118
:10264000939F500D112470E0CA010E9498266038B3
:10265000710540F46115710519F406C068E070E079
:10266000862F08958FE7089581E0089580913A02BA
:1026700080FF08C06091050170E0759567957595BC
:10268000679521C081FF06C06091050170E07595D6
:10269000679519C082FF04C06091050170E010C009
:1026A00090913802992399F0609104019617A0F750
:1026B00080910501899FC001112470E00E94982635
:1026C0006038710540F46115710519F406C061E0C8
:1026D00070E0862F08958FE7089581E008958D3E7C
:1026E00021F40E94F712819504C08E3E29F40E94C5
:1026F000F71280933E0208958F3E21F40E94F71254
:10270000819504C0803F29F40E94F71280933D0216
:102710000895893F19F40E94361305C08A3F31F4A9
:102720000E943613819580933F0208958B3F21F4D8
:102730000E943613819504C08C3F29F40E94361301
:102740008093400208959FE0980F983078F421E03C
:1027500030E0A90102C0440F551F9A95E2F7CA0163
:1027600090913C02892B80933C0208958D3F21F487
:1027700080913A0281600BC08E3F21F480913A0231
:10278000826005C08F3F29F480913A028460809373
:102790003A0208958D3E39F490913E0297FF35C07C
:1027A00010923E0259C08E3E29F490913E021916B5
:1027B000BCF32BC090913D028F3E29F497FF25C0BA
:1027C00010923D0249C0803F19F41916CCF31DC088
:1027D00090913F02893F29F41916BCF410923F02F0
:1027E0003BC08A3F19F497FF10C0F8CF8B3F39F4F4
:1027F0009091400297FF09C0109240022DC08C3F7B
:1028000021F4909140021916BCF39FE0980F983084
:1028100080F421E030E0A90102C0440F551F9A95D1
:10282000E2F7CA01809590913C02892380933C0293
:1028300013C08D3F21F480913A028E7F0BC08E3FF2
:1028400021F480913A028D7F05C08F3F29F4809159
:102850003A028B7F80933A0280913D02811106C03B
:1028600080913E02811102C01092390280913F0294
:10287000811106C080914002811102C0109238027D
:1028800008950E94671F20913D02211104C02091EC
:102890003E02222321F0909337028093360220914A
:1028A0003F02211104C020914002222321F0909385
:1028B0003502809334028BE392E00C948C1EEF92ED
:1028C000FF920F931F93CF93DF9300D000D000D0DF
:1028D000CDB7DEB786E0EBE3F2E0DE0111960190C2
:1028E0000D928A95E1F7E0903D02F0903E02009152
:1028F0003F021091400210923D0210923E0210924F
:102900003F0210924002E11003C0FF2009F45DC0B5
:1029100080913602909137020E947F1FAC01909106
:102920003902992339F020910A0130E02417350744
:1029300058F04BC020910B018AE0289F9001112490
:102940002417350718F041C09F3F19F09F5F9093FF
:102950003902EE2061F00E94F7121E1414F09FEF6E
:1029600001C091E0989F902D112490933D02FF208B
:1029700061F00E94F7121F1414F09FEF01C091E064
:10298000989F902D112490933E0230913D02332365
:10299000E1F020913E022223C1F045EB3403C00157
:1029A0001124992319F090933D0203C081E0809394
:1029B0003D0235EB2303C0011124992319F09093B4
:1029C0003E0203C081E080933E02011103C0112347
:1029D00009F45DC080913402909135020E947F1FFE
:1029E000AC0190913802992339F02091060130E032
:1029F0002417350758F04BC0209107018AE0289F23
:102A0000900111242417350718F041C09F3F19F099
:102A10009F5F90933802002361F00E9436131016D6
:102A200014F09FEF01C091E0989F902D1124909396
:102A30003F02112361F00E943613111614F09FEF2C
:102A400001C091E0989F902D112490934002309105
:102A50003F023323E1F0209140022223C1F045EBF5
:102A60003403C0011124992319F090933F0203C04D
:102A700081E080933F0235EB2303C00111249923A9
:102A800019F09093400203C081E08093400280914E
:102A90003D0281110BC080913E02811107C08091DF
:102AA0003F02811103C08091400281110E944114B4
:102AB000EB82FC820D831E8386E0FE013196ABE340
:102AC000B2E001900D928A95E1F726960FB6F89440
:102AD000DEBF0FBECDBFDF91CF911F910F91FF9051
:102AE000EF900895EBE3F2E086E0DF011D928A9516
:102AF000E9F7109239021092380210923A020895C2
:102B0000CF93DF93EC01FB018281882309F43CC160
:102B1000C430FDE5DF0760F4CB3F9CE5D90788F4BE
:102B20009E0122503C452431310508F02EC109C0D8
:102B3000C236EDE5DE0729F0C63AFDE5DF0709F00C
:102B400024C10E94D80D9093020480930104C131E6
:102B50008CE5D80709F4C6C008F042C0C930ECE5DE
:102B6000DE0709F49BC000F5C5308CE5D80709F4F1
:102B700085C078F4C330ECE5DE0709F478C008F0CE
:102B80007AC0C230DC4509F0F5C080910104816053
:102B9000EFC0C7309CE5D90709F478C008F07AC0C7
:102BA000809101048061E4C0CD30FCE5DF0709F4C9
:102BB00087C058F4CB309CE5D90709F479C008F0F8
:102BC0007BC08091010488606FC0CF30FCE5DF07D7
:102BD00009F480C008F082C080910104877FC8C0DA
:102BE000CE3F9CE5D90709F471C000F5C531FCE57D
:102BF000DF0709F485C068F4C3319CE5D90709F4FF
:102C000075C008F095C00E948F07809101048F77EE
:102C1000AFC0CC3FFCE5DF07A9F108F054C0CB3FC3
:102C2000DC4509F0A7C08091020440C0C230EDE548
:102C3000DE0709F489C058F4C1158DE5D80709F4F9
:102C40005AC008F069C08091020482602FC0C23669
:102C5000EDE5DE0709F47CC0C63AFDE5DF0709F4BF
:102C600081C0C330DD4509F085C080E06EC0809131
:102C7000010482607DC08091010416C0809101042E
:102C8000886076C08091020482604FC08091010408
:102C900080626EC08091010480646AC00E948F07C8
:102CA00080910104806864C0846062C081603DC01E
:102CB000809101048E7F5CC0809101048D7F58C09B
:102CC0008091010416C08091020418C08091020412
:102CD0008D7F2BC0809101048F7E4AC080910104BA
:102CE0008F7D46C0809101048F7B42C0809101049A
:102CF000877F8B7F3DC0809102048D7F8E7F15C0C2
:102D00008091010482FB222720F991E0922790FB19
:102D100082F990FB83F92CC080910204982F909542
:102D200091708E7F892B90FB81F98093020422C0E1
:102D30000E948F078091010487FB222720F991E0F0
:102D4000922790FB87F914C081E00E946F0E12C099
:102D50008091010484FB222720F991E0922790FBC7
:102D600084F906C080910104982F909590FB80F91A
:102D70008093010480910104909102040E94E90D66
:102D80000E948F0780E001C081E0DF91CF9108951C
:102D90000895CF93C82F0E94C816C0934102CF91C7
:102DA00008950E949226811104C00E94931A83E024
:102DB000089582E0089580914102811102C00C942F
:102DC000D1160895873941F178F4863349F130F40A
:102DD000843321F1853331F584E208958439D1F0CB
:102DE000863901F581E20895843F71F030F4803F27
:102DF000D9F0813FB9F481E00895863F49F030F081
:102E0000873F81F487E0089584E0089585E0089580
:102E100086E0089580E2089582E2089583E20895AD
:102E200085E208958FE1089580E0089595E89093F4
:102E30007A00982F9072906890937B008F71909198
:102E40000C01892B80937C0080917A0080648093B0
:102E50007A0080917A0086FDFCCF809178002091E5
:102E6000790090917A009F7790937A0090E0922B6E
:102E700008950E94E2160C941617EF92FF920F939A
:102E80001F93CF93DF93EC018B0122E030E040E011
:102E900060E084E30E946A1D0E94671F7C018881B4
:102EA0000E94E31D8E3F9105A9F40E94431E82E417
:102EB0008A95F1F700C022E030E040E060E084E372
:102EC0000E946A1DC7010E947F1F8017910738F377
:102ED000C0E00AC06B816F7770E06D5F7F4FCE01FD
:102EE00001960E94131EC1E00E94431E8C2FDF91A9
:102EF000CF911F910F91FF90EF900895EF92FF9265
:102F00000F931F93CF93DF93EC017B010E94671F08
:102F10008C0166990CC082E08A95F1F700C0C80167
:102F20000E947F1F8E159F05A0F3C0E035C022E0F0
:102F300030E040E060E084E30E946A1D0E94FB1DD7
:102F400088838E5F8230A8F40E94431E82E48A95B3
:102F5000F1F700C022E030E040E060E084E30E944E
:102F60006A1DC8010E947F1F8E159F0538F3C0E0BF
:102F700011C063E070E0CE0101960E942B1E6B81B0
:102F80006F7770E06131710524F4CE0104960E94E0
:102F90002B1EC1E00E94431E8C2FDF91CF911F9109
:102FA0000F91FF90EF9008951F93CF93DF93CDB7CC
:102FB000DEB764970FB6F894DEBF0FBECDBFE091C9
:102FC000470290914602E91709F43FC0182F669B0B
:102FD00021C066E970E0CE0101960E947E17882329
:102FE000A1F18C8187FD0DC020914702809146029E
:102FF000281759F130E02F5F3F4F2170332720937E
:103000004702112311F190914702809146029813D3
:103010001AC01BC0F0E0EE0FFF1FEE5BFD4F80817A
:1030200091810E947F1F8D32914078F080914702FC
:1030300090914602891749F090E001968170992796
:103040008093470202C06699C4CF64960FB6F89485
:10305000DEBF0FBECDBFDF91CF911F9108956F925C
:103060007F928F929F92AF92BF92CF92DF92EF9218
:10307000FF920F931F93CF93DF93CDB7DEB7A8973F
:103080000FB6F894DEBF0FBECDBF7C018B016A0185
:103090004901FC0101900020E9F7CF0101975C0193
:1030A000672B61F09091460280914702981721F0BA
:1030B00081E00E94D417F6CFF801108240E1742E0F
:1030C0005AE0652EA5014E195F09888D41315105E1
:1030D000DCF07D8A1E8A6F8A807880618068888FA4
:1030E000F701DE015996872D01900D928A95E1F73F
:1030F000B401CE0145960E943D17882309F464C0AF
:10310000F0E1EF0EF11CDECF80E18D8B1E8A8AE0AC
:103110008F8B842F8F77888F5527B701CE014996E3
:103120000E941327B401CE0145960E943D17F82E48
:10313000882309F449C001151105E1F40E94671FB5
:103140008C018091460290E09C012F5F3F4F2170DF
:10315000332740914702421709F45AC0880F991F3C
:10316000FC01EE5BFD4F11830083209346020E9419
:10317000671F52C05801AC0CBD1C78016CE271E0B5
:10318000CE0101960E947E178823F1F0898180325A
:1031900019F0F801108218C08C818F77CA2CCE18D4
:1031A0008C1508F4C82ECC2051F0D12CA601BE01FC
:1031B0006B5F7F4FC7010E941327EC0CFD1C8C81B5
:1031C00087FDDCCFF70106C0F12C26C07F0180818E
:1031D0008A3039F41082F70131970E171F07B0F3C8
:1031E00002C08D30B9F36AE070E0C8010E94272761
:1031F000009719F08C010F5F1F4F65E173E0C80164
:103200000E94ED2621E0892B09F020E0F22E04C077
:1032100080E00E94D41795CF8F2DA8960FB6F89412
:10322000DEBF0FBECDBFDF91CF911F910F91FF90F9
:10323000EF90DF90CF90BF90AF909F908F907F9056
:103240006F9008958F929F92AF92BF92CF92DF922C
:10325000EF92FF920F931F93CF93DF93CDB7DEB71B
:103260007C015B014A01CDB6DEB60E94FD260196C7
:103270002DB73EB7281B390B0FB6F8943EBF0FBED3
:103280002DBF0DB71EB70F5F1F4FB701C8010E94BA
:10329000F62626E930E0A401B501C8010E942F18E6
:1032A0000FB6F894DEBE0FBECDBEDF91CF911F9159
:1032B0000F91FF90EF90DF90CF90BF90AF909F90D5
:1032C0008F9008958F929F92AF92BF92CF92DF928C
:1032D000EF92FF920F931F93CF93DF93CDB7DEB79B
:1032E000CA57D1090FB6F894DEBF0FBECDBF7C011F
:1032F0009091460280914702981301C19091D903A1
:103300008091D803981709F4FAC08AE0899F900148
:103310001124285B3D4FF901DE01AF58BF4F0190EA
:103320000D928A95E1F7F901C08015810681D78059
:10333000908481840E94671F9093E5038093E40347
:10334000F1E0CF1679F1CF1628F022E0C21609F489
:1033500052C0BAC068EA72E0CE0101965C010E94D8
:10336000F6261F928F921F929F921F92DF921F92BA
:103370000F931F921F93E6968FADE6971F928F9340
:10338000E5968FADE5971F928F93BF92AF921F92F4
:1033900080E38F938E010F5B1F4F1F930F930E944B
:1033A0003A271BC06DE872E08E010F5F1F4FC80106
:1033B0000E94F626E6968FADE6978F93E5968FAD41
:1033C000E5978F931F930F931F9280E38F93005C79
:1033D0001F4F1F930F930E943A27970140E050E040
:1033E00060E070E0C8010E942F180FB6F894DEBFAD
:1033F0000FBECDBF67C06EE672E0CE0101965C01E4
:103400000E94F626802F002E000C990B9F930F939D
:10341000812F012E000C990B9F931F93E6968FAD81
:10342000E697282F082E000C330B3F938F93E596D9
:103430008FADE597282F082E000C330B3F938F9309
:10344000BF92AF921F9280E38F938E010F5B1F4F4D
:103450001F930F930E943A27970140E050E060E0ED
:1034600070E0C8010E942F180FB6F894DEBF0FBE9F
:10347000CDBF8823C1F168E572E0C8010E94F6263D
:10348000D0FE05C06DE871E0C8010E941C27D1FE86
:1034900005C06FE871E0C8010E941C27D2FE03C07E
:1034A00061E971E004C0D11005C063E971E0C801B1
:1034B0000E941C27970140E050E060E070E0C801E6
:1034C0000E942F18882379F08091D9039091D80316
:1034D0008917A9F090E0019668E270E00E949826B2
:1034E0008093D9030CC0FFE729EA33E0F150204074
:1034F0003040E1F700C0000081E00E94D417C658B8
:10350000DF4F0FB6F894DEBF0FBECDBFDF91CF9176
:103510001F910F91FF90EF90DF90CF90BF90AF90F1
:103520009F908F9008958091DA0308950F931F93D1
:10353000CF93DF93CDB7DEB7C258D1090FB6F89459
:10354000DEBF0FBECDBF8091DB0381111EC0109284
:10355000DC031092DA036E9876980E94621D549AEA
:103560005C9A5C988FE19EE40197F1F700C000003F
:103570005C9A9FEF29E688E1915020408040E1F776
:1035800000C0000081E08093DB031092DC030EE6B4
:1035900013E042E050E0B801CE018F579F4F0E94E8
:1035A000E42640E850E0BE016F5F7F4FCF57DF4F0A
:1035B00088819981C158D0400E942219882379F0CE
:1035C0000E5F1F4F93E00A37190719F781E08093C8
:1035D000DC030E94671F9093E5038093E4038091CE
:1035E000DC03CE57DF4F0FB6F894DEBF0FBECDBF62
:1035F000DF91CF911F910F910895CF93DF93CDB7B6
:10360000DEB7E0970FB6F894DEBF0FBECDBF809156
:10361000DC03811105C00E94961A882309F46DC04D
:1036200081E00E94D4178AE090E00E9462198091A4
:10363000E4039091E5030E947F1F893E9340C8F107
:103640008091DD03811117C040E350E0BE016F5F40
:103650007F4F82E093E00E942219882349F040E3E3
:1036600050E0BE016F5F7F4F8FEE92E00E94221903
:1036700081E08093DD030E94671F9093E5038093B0
:10368000E40340E350E0BE016F5F7F4F81EE92E0C4
:103690000E942219882369F0CE0101960E94C62655
:1036A00021E0892B09F420E08091DA038213209332
:1036B000DA038091DE039091DF030E947F1F813146
:1036C0009742D8F09091460280914702981315C016
:1036D0000E94671F9093DF038093DE0385E30E94BF
:1036E0003917092E000CAA0BBB0B8093E0039093B3
:1036F000E103A093E203B093E303E0960FB6F894DE
:10370000DEBF0FBECDBFDF91CF9108950F931F9302
:10371000CF93DF93EC01FB018C0100571E4FD801C2
:103720002C9130E0C901019668E270E00E94982671
:10373000DE01AF56BE4F9C91981781F09AE0929FA0
:10374000D001939FB00D1124AC0FBD1F01900D92BD
:103750009A95E1F7F801808381E001C080E0DF9174
:10376000CF911F910F910895FF920F931F93CF93C5
:10377000DF93CDB7DEB72A970FB6F894DEBF0FBE42
:10378000CDBF8B01F42E19828C830E94671F9B830F
:103790008A83F80180818D83FF2011F0818101C02F
:1037A00080E08E83F1E0FF1518F4F801828101C0FA
:1037B00080E08F83F2E0FF1518F4F801838101C0E7
:1037C00080E08887F3E0FF1518F4F801848101C0D8
:1037D00080E08987F4E0FF1518F4F801858101C0C5
:1037E00080E08A87BE016F5F7F4F88E492E00E948D
:1037F000861B811105C086E990E00E946219C9CF3D
:10380000F6E0FF1528F48AEFF80E0A5F1F4FC1CFCC
:103810002A960FB6F894DEBF0FBECDBFDF91CF91D1
:103820001F910F91FF900895CF93DF93CDB7DEB72F
:103830002A970FB6F894DEBF0FBECDBF21E02983D3
:103840009D838C83BE016F5F7F4F88E492E00E946E
:10385000861B811105C086E990E00E946219F2CFB3
:103860002A960FB6F894DEBF0FBECDBFDF91CF9181
:1038700008950F93CF93DF93CDB7DEB72A970FB696
:10388000F894DEBF0FBECDBF92E099838C836D8329
:103890004E832F830887BE016F5F7F4F88E492E0DD
:1038A0000E94861B811105C086E990E00E94621982
:1038B000F2CF2A960FB6F894DEBF0FBECDBFDF91D0
:1038C000CF910F9108951092D8031092D903E2E49A
:1038D000F2E0148215820895CF93DF9386319C45E0
:1038E00041F5EB010E94E20C982F8A8120910201A0
:1038F00030910301882379F09A7A81E009F480E01D
:103900008093E603911102C069E201C065E3C90139
:103910000E94081F0AC08091E603811102C069E27B
:1039200001C065E3C9010E940A1F0E94240D80E0C6
:1039300001C081E0DF91CF9108950F931F93CF9342
:10394000DF93C42FD22FFC0182818823C9F04093DA
:10395000E9030E94671F9093E8038093E70380E2E6
:103960008C0F883008F057C0C77081E001C0880F05
:10397000CA95EAF7DF91CF911F910F910C94EC0457
:103980008091E903481330C08091E7039091E803E8
:103990000E947F1F8436910538F510E21D0FCD1768
:1039A000B9F080E28C0F883040F4C77081E001C02C
:1039B000880FCA95EAF70E94F304183028F581E0D1
:1039C0009D2F977001C0880F9A95EAF70E94EC042A
:1039D000802F0E94E3041830F0F4D77081E001C01A
:1039E000880FDA95EAF70AC080E28C0F883098F4E5
:1039F000C77081E001C0880FCA95EAF7DF91CF91C7
:103A00001F910F910C94F304802FDF91CF911F91A0
:103A10000F910C94E304DF91CF911F910F910895C2
:103A20000F939C01CB01243F4CE5340731F188F41E
:103A3000293DFCE53F07D9F02A3D4CE5340779F1F3
:103A4000283D3C45A9F506E221EE41EE68ED7CE516
:103A50002BC0263FFCE53F07E1F0A8F0273F3C459F
:103A600039F507E225EE46EE67EF7CE51DC007E27B
:103A700025EE45EE69ED7CE517C006E221EE40EE4D
:103A800064EF7CE511C007E225EE44EE65EF7CE5CE
:103A90000BC006E221EE42EE66EF7CE505C008E2CF
:103AA00021E045EE6AED7CE50E949D1C80E008C0A7
:103AB000FC018281882319F01092E90301C081E0A2
:103AC0000F910895289A219A229A23982B9880E59D
:103AD0008CBD089590910D019F3F09F072C08F3FFA
:103AE00009F46FC0611103C01092EB0303C090E2B0
:103AF0009093EB03423041F0433051F0413069F490
:103B00009091EB03946007C09091EB03986003C021
:103B10009091EB039C609093EB0341E050E04217DF
:103B2000530718F4440F551FFACF9091EB0340311F
:103B30005105F1F050F442305105B1F048305105D3
:103B4000E1F421E02093EA0313C04034510591F0E1
:103B50004038510539F04032510579F421E0209385
:103B6000EA0308C0936007C091E09093EA0305C0A0
:103B7000916001C092609093EB032CB59091EB03A0
:103B8000922B9CBD9091EA03992319F09DB5916009
:103B90009DBD80930D01E82FE295EF70F0E031A11B
:103BA000282F2F7081E090E001C0880F2A95EAF756
:103BB000932F982B91A392A18095892382A381E0D2
:103BC000089580E00895CF93DF938EBD0E94671F14
:103BD000EC010DB407FC0AC00E94671F8C1B9D0BF3
:103BE00084369105B0F38EEF9FEF02C08EB590E062
:103BF000DF91CF910895CF93DF931EBC0E94671F82
:103C0000EC010DB407FC0AC00E94671F8C1B9D0BC2
:103C100084369105B0F38EEF9FEF02C08EB590E031
:103C2000DF91CF9108950F931F93CF93DF93EC0112
:103C30008C01060F171FC017D10731F089910E9420
:103C4000E31D97FD03C0F7CF80E090E0DF91CF91B7
:103C50001F910F9108950F931F93CF93DF93EC0162
:103C60008C01060F171FC017D10731F00E94FB1DF2
:103C700097FD04C08993F7CF80E090E0DF91CF916A
:103C80001F910F91089580910D018F3F19F1E82F39
:103C9000E295EF70F0E031A1282F2F7081E090E0E5
:103CA00001C0880F2A95EAF7932F982B91A392A130
:103CB000892B82A38FEF80930D018DB58E7F8DBDF3
:103CC0009CB58091EB03809589238CBD1092EB030A
:103CD0001092EA0308959093AB018093AA0108958E
:103CE0009093F1038093F0030895E091F003F09135
:103CF000F103309721F00190F081E02D099480E0EC
:103D00000895E091F003F091F103309721F00280E3
:103D1000F381E02D09940895E091F003F091F1030F
:103D2000309739F022E0DC012C930480F581E02DFE
:103D3000099408952091EE033091EF032817390775
:103D400071F09093EF038093EE03E091F003F09114
:103D5000F103309721F00680F781E02D0994089552
:103D60002091EC033091ED032817390771F09093FF
:103D7000ED038093EC03E091F003F091F1033097B1
:103D800021F00084F185E02D09940895FC0132961C
:103D900097E080E0915029F021912223D9F38F5FA1
:103DA000F9CF0895662349F0FC01329608962191D7
:103DB000621729F0E817F907D1F780E0089581E04C
:103DC00008959C01FC0132969FEF80E041914617D7
:103DD00089F09F3F19F4411101C0982F8F5F863001
:103DE000A9F79F3F39F0F901E90FF11D97FDFA9509
:103DF0006283089508959C012A5F3F4FFC01428130
:103E0000461301C01282019682179307B9F70895ED
:103E10000C94E11E0C94FB1E029626E0FC0111920C
:103E20002A95E9F7089508950C94131F83E0809371
:103E3000F2030C94141F811102C081E001C082E0E2
:103E40008093F2030C94141F0C941B1F81E0809349
:103E5000F2030C94141F0C94261F08950C942D1F2C
:103E600008951F920F920FB60F9211248F939F9374
:103E7000AF93BF938091F303811113C0809113041A
:103E800090911404A0911504B09116044196A11DBF
:103E9000B11D8093130490931404A0931504B09360
:103EA0001604BF91AF919F918F910F900FBE0F900D
:103EB0001F9018950E948F070C94460382E084BDE2
:103EC00093E095BD9DE797BD80936E0008952FB751
:103ED000F8948091130490911404A0911504B0916A
:103EE00016042FBF08952FB7F894609113047091B2
:103EF000140480911504909116042FBF08959C011D
:103F00004FB7F8948091130490911404A091150474
:103F1000B09116044FBF821B930B089578941F92A3
:103F20000F920FB60F9211248F939F93AF93BF936D
:103F30008091130490911404A0911504B09116047B
:103F40000196A11DB11D8093130490931404A093B6
:103F50001504B0931604BF91AF919F918F910F906C
:103F60000FBE0F901F90189587E797E79093010871
:103F7000809300089AE088E10FB6F894A8958093A2
:103F800060000FBE90936000FFCF8091FF03089503
:103F900008950F93CF93DF93EC010E94DB168330DB
:103FA00041F409812D814C816B818A810E94391CE9
:103FB0001FC082E08093E9008FEF9091E80081506C
:103FC00095FD06C09AE69A95F1F700C08111F5CFEC
:103FD0008091E80085FF0CC040E050E066E070E0B2
:103FE000CE010E94F7218091E8008E778093E8004F
:103FF000DF91CF910F910895CF93DF93EC010E9451
:10400000DB16833049F4BE016E5F7F4F46E0888146
:10401000DF91CF910C94B41B81E08093E9008FEF86
:104020009091E800815095FD06C09AE69A95F1F7C7
:1040300000C08111F5CF8091E80085FF14C040E0F9
:1040400050E068E070E0CE010E94F7218091E80026
:104050008E778093E80088E0FE01A7EFB3E001903F
:104060000D928A95E1F7DF91CF9108958093F40343
:104070007093F6036093F50380911B04843001F57F
:1040800082E08093E9008FEF9091E800815095FDE8
:1040900006C09AE69A95F1F700C08111F5CF80919C
:1040A000E80085FF0DC040E050E063E070E084EF81
:1040B00093E00E94F7218091E8008E778093E800DA
:1040C0000895CF93DF93EC010E94DB16833029F42F
:1040D000CE01DF91CF910C94141CBE0184E0DF91DE
:1040E000CF910C943620BC0183E00C943620809153
:1040F0001A04811109C00E9488230E94E52380913F
:10410000E20084608093E200089510921A040895FA
:104110000C942B1F6091170481E0611101C080E0B5
:104120000C94161F0E945A1F90911B0481E094303A
:1041300009F080E0609117040C941B1F42E061ECD1
:1041400081E00E94012342E261EC82E00E940123AF
:1041500090911B0481E0943009F080E06091170495
:104160000C94241F80911D04833009F461C030F445
:10417000813071F0823009F49AC008958A3009F4D0
:1041800086C08B3009F46CC0893009F0A8C020C00B
:1041900080911C04813A09F0A2C08091E800877FD9
:1041A0008093E8008091200490912104892B21F4D0
:1041B00068E087EF93E003C060E080E090E070E0AB
:1041C0000E9442228091E8008B778093E800089556
:1041D00080911C04813209F082C08091200490916A
:1041E0002104029708F07BC08091E800877F8093CC
:1041F000E8008091E80082FD05C080911B048111D8
:10420000F8CF6DC02091F3008091F20090E0922BE6
:10421000029731F48091F100813011F0863021F461
:104220008091F1008093FF038091E8008B7753C069
:1042300080911C04813A09F052C080912004909131
:104240002104892B09F04BC08091E800877F80937F
:10425000E8008091E80080FFFCCF80911A0136C011
:1042600080911C048132D9F5809120049091210421
:10427000892BA9F58091E800877F8093E8000E9450
:10428000362380911E0480931A010C948F0780912D
:104290001C04813221F58091E800877F8093E8003B
:1042A0000E94362380911F0480930004089580911A
:1042B0001C04813AA1F48091E800877F8093E80094
:1042C0008091E80080FFFCCF809100048093F10092
:1042D0008091E8008E778093E8000C94362308954F
:1042E00084B7877F84BF0FB6F894A895809160004B
:1042F000886180936000109260000FBE90E080E8BB
:104300000FB6F89480936100909361000FBE0C94F7
:10431000261F0E9488230E94E523E2EEF0E08081C0
:104320008460808378940C9477268EE091E00C94DE
:10433000701E08950C94FD1A0C949E21292F33278A
:1043400023303105C9F060F42130310581F022308D
:10435000310509F044C08BE390E026E933E043C027
:1043600021323105E1F02232310549F138C082E1D4
:1043700090E021ED33E037C099278130910549F075
:1043800028F0029761F5EAE7F3E005C0E2E9F3E01F
:1043900002C0E2E8F3E0849190E09F0124C061153F
:1043A000710541F061307105D1F489E090E021ECB4
:1043B00033E019C089E090E028EA33E014C06115C9
:1043C000710541F06130710551F48BE790E023EE07
:1043D00033E009C080E490E02EE534E004C080E0E2
:1043E00090E020E030E0FA01318320830895CF92FD
:1043F000DF92EF92FF920F931F93CF93DF93EC0125
:104400008B017A010E945523811133C0E114F1041C
:1044100039F0F70180819181081B190BC80FD91F52
:10442000C12CD12C0115110519F18091E80085FDF1
:1044300016C08091E8008E778093E800E114F104C3
:1044400049F0F70180819181C80ED91ED182C082C6
:1044500085E00FC00E945523882321F30AC089916B
:104460008093F10001501109FFEFCF1ADF0ADACF74
:1044700080E0DF91CF911F910F91FF90EF90DF903F
:10448000CF900895209122043091230426173707F6
:1044900048F06115710539F42091E8002E772093DA
:1044A000E80001C0B901FC0120E06115710579F156
:1044B00080911B048823F1F18530F1F18091E800AF
:1044C00083FD3CC08091E80082FD2EC08091E80011
:1044D00080FFEBCF2091F3008091F20090E0922BCF
:1044E0006115710551F08830910538F421912093C0
:1044F000F100615071090196F3CF21E0089709F0AE
:1045000020E08091E8008E778093E800CECF2111E3
:10451000CFCF0AC080911B04882361F0853061F001
:104520008091E80083FD0AC08091E80082FFF2CF0D
:1045300080E0089582E0089583E0089581E0089581
:1045400020912204309123042617370748F0611583
:10455000710539F42091E8002E772093E80001C01E
:10456000B901FC0120E06115710591F180911B04F6
:10457000882309F440C0853009F43FC08091E800E9
:1045800083FD3DC08091E80082FD2FC08091E8004E
:1045900080FFE9CF2091F3008091F20090E0922B10
:1045A0006115710559F08830910540F424912093EC
:1045B000F1003196615071090196F2CF21E0089720
:1045C00009F020E08091E8008E778093E800CBCF5F
:1045D0002111CCCF0AC080911B04882361F0853063
:1045E00061F08091E80083FD0AC08091E80082FFBD
:1045F000F2CF80E0089582E0089583E0089581E09D
:104600000895982F973068F59093E900981739F03E
:104610007091EC002091ED005091F00003C0242F28
:10462000762F50E021FD02C09F5FECCF3091EB0070
:104630003E7F3093EB003091ED003D7F3093ED00F5
:104640003091EB0031603093EB007093EC002093DD
:10465000ED005093F0002091EE0027FDE5CF80E0C3
:1046600008958F708093E90081E0089580911C0483
:1046700087FF11C08091E80082FD05C080911B0476
:104680008111F8CF11C08091E8008B770BC0809129
:104690001B04882349F08091E80080FFF8CF8091C7
:1046A000E8008E778093E80008952091E40030912F
:1046B000E50095E64091EC00842F817040FF23C017
:1046C0008091E80080FD1DC080911B04882399F033
:1046D000853099F08091EB0085FD11C04091E40098
:1046E0005091E5002417350729F3915011F09A01F4
:1046F000E1CF84E0089582E0089583E0089581E0A9
:10470000089580E008954091E80042FFDDCF0895CC
:104710000E94F6230E94FE23E0EEF0E0808181609B
:104720008083E8EDF0E080818F77808319BCA7ED6E
:10473000B0E08C918E7F8C9380818F7E80831092ED
:104740001A0408950F931F93CF93DF930E94F623CB
:104750000E94FE23C8EDD0E088818F77888388810E
:104760008068888388818F7D888319BC10921B04A0
:1047700010921704109219041092180400EE10E021
:10478000F80180818B7F808388818160888342E00B
:1047900060E080E00E940123E1EEF0E080818E7F06
:1047A0008083E2EEF0E08081816080838081886098
:1047B0008083F80180818E7F8083888180618883F7
:1047C000DF91CF911F910F910895E8EDF0E0808186
:1047D0008F7E8083E7EDF0E080818160808384E0DC
:1047E00082BF81E080931A040C94A223E8EDF0E0EC
:1047F00080818E7F80831092E20008951092DA000B
:104800001092E10008951F920F920FB60F9211249B
:104810002F933F934F935F936F937F938F939F93C8
:10482000AF93BF93EF93FF938091E10082FF0BC0A2
:104830008091E20082FF07C08091E1008B7F80932E
:10484000E1000E9476268091DA0080FF1DC08091F1
:10485000D80080FF19C08091DA008E7F8093DA0043
:104860008091D90019BC80FF0BC082E089BD09B4DA
:1048700000FEFDCF81E080931B040E94772004C0DE
:1048800010921B040E9485208091E10080FF19C0D6
:104890008091E20080FF15C08091E2008E7F8093BE
:1048A000E2008091E20080618093E2008091D80074
:1048B00080628093D80019BC85E080931B040E941D
:1048C0008A208091E10084FF2FC08091E20084FF64
:1048D0002BC019BC82E089BD09B400FEFDCF8091D8
:1048E000D8008F7D8093D8008091E1008F7E8093E7
:1048F000E1008091E2008F7E8093E2008091E200EF
:1049000081608093E20080911704882311F084E095
:1049100007C08091E30087FD02C081E001C083E011
:1049200080931B040E9492208091E10083FF29C0A4
:104930008091E20083FF25C08091E100877F809312
:10494000E10082E080931B04109217048091E10043
:104950008E7F8093E1008091E2008E7F8093E20061
:104960008091E20080618093E20042E060E080E0BC
:104970000E9401238091F00088608093F0000E94E3
:104980008820FF91EF91BF91AF919F918F917F917F
:104990006F915F914F913F912F910F900FBE0F90AC
:1049A0001F9018951F920F920FB60F9211242F93FC
:1049B0003F934F935F936F937F938F939F93AF93A7
:1049C000BF93CF93DF93EF93FF93C091E900CF7034
:1049D0008091EC00D82FD17080FDD0E81092E900D2
:1049E0008091F000877F8093F00078940E941625D4
:1049F0001092E9008091F00088608093F000CD2B48
:104A0000CF70C093E900FF91EF91DF91CF91BF91FB
:104A1000AF919F918F917F916F915F914F913F9156
:104A20002F910F900FBE0F901F9018951F93CF934B
:104A3000DF93CDB7DEB7AA970FB6F894DEBF0FBEEF
:104A4000CDBFECE1F4E08091F100819324E0E43209
:104A5000F207C9F70E94B2208091E80083FF2EC1BF
:104A600080911C0490911D04492F50E04A3051055B
:104A700008F024C1FA01EE59FF4F0C94AC2680389F
:104A800021F0823809F01AC108C080911804909171
:104A90001904992389F082600FC0809120048F70DF
:104AA000873008F00BC18093E9008091EB0085FB13
:104AB000882780F91092E9009091E800977F909301
:104AC000E8008093F1001092F100D1C0282F2D7FD3
:104AD00009F0F4C0882319F0823061F0EFC08091B2
:104AE0001E04813009F0EAC0933009F080E0809321
:104AF00019042EC080911E0481112AC080912004C7
:104B00008F702FEF280F263008F0D8C08093E9006F
:104B10002091EB0020FF1CC0933021F48091EB002A
:104B2000806214C09091EB0090619093EB0021E0C3
:104B300030E0A90102C0440F551F8A95E2F7409367
:104B4000EA001092EA008091EB0088608093EB000D
:104B50001092E9008091E800877F8093E8000E942E
:104B60003623ACC08111AAC010911E041F7780911A
:104B7000E3008078812B8093E3008091E800877FB9
:104B80008093E8000E9436238091E80080FFFCCFEC
:104B90008091E30080688093E300111102C082E0FD
:104BA00001C083E080931B0489C08058823008F0E4
:104BB00085C080911E0490911F048C3D53E09507A1
:104BC00079F583E08A838AE289834FB7F894DE011E
:104BD000139620E03EE051E2E32FF0E050935700BF
:104BE000E49120FF03C0E295EF703F5FEF708E2FDE
:104BF00090E0EA3010F0C79601C0C0968D939D9367
:104C00002F5F243149F74FBF8091E800877F809361
:104C1000E8006AE270E0CE0101960E94422216C0CE
:104C20006091200470912104AE014F5F5F4F0E949C
:104C30009C21BC01892B09F441C09091E800977F29
:104C40009093E80089819A810E94A0228091E800D7
:104C50008B778093E80032C0803881F58091E8003E
:104C6000877F8093E800809117048093F100809102
:104C7000E8008E7772CF811121C080911E0490913F
:104C80001F0499270297D4F48091E800877F8093CE
:104C9000E80080911E04809317040E9436238091BF
:104CA0001704811106C08091E30087FD02C081E0F6
:104CB00001C084E080931B040E949E208091E80044
:104CC00083FF0AC08091E800877F8093E80080918D
:104CD000EB0080628093EB00AA960FB6F894DEBFDB
:104CE0000FBECDBFDF91CF911F9108950895CF934F
:104CF00080911B048823A1F0C091E900CF709091AE
:104D0000EC00892F817090FD80E8C82B1092E9009B
:104D10008091E80083FD0E941625CF70C093E900C2
:104D2000CF9108958091E300881F8827881F0895F8
:104D300097FB072E16F4009407D077FD09D00E9448
:104D4000B22607FC05D03EF4909581959F4F0895BB
:104D5000709561957F4F0895EE0FFF1F0590F491B8
:104D6000E02D0994AA1BBB1B51E107C0AA1FBB1F62
:104D7000A617B70710F0A61BB70B881F991F5A95E7
:104D8000A9F780959095BC01CD010895FC01882775
:104D90009927E89421912032E9F3293010F02E3040
:104DA000C8F32B3241F02D3239F4689404C00E94CC
:104DB0003227820F911D219120532A30C0F31EF417
:104DC000909581959F4F0895FB01DC0102C00590ED
:104DD0000D9241505040D8F70895FB01DC018D91B0
:104DE000059080190110D9F3990B0895FB01DC019E
:104DF00005900D920020E1F70895FC010590002038
:104E0000E9F7809590958E0F9F1F0895FB01DC01B7
:104E100004C08D910190801921F441505040C8F791
:104E2000881B990B0895FB01DC0102C001900D92D3
:104E300041505040D8F70895FB01DC010D9000204F
:104E4000E9F7119701900D920020E1F70895FC0118
:104E500081E090E00190061609F4CF010020D1F71F
:104E6000019708957AE0979F902D879F802D910D4F
:104E700011240895AEE0B0E0E0E4F7E20C944B2A90
:104E80000D891E898F89988D26E02C831A830983CA
:104E900097FF02C080E090E801979E838D83AE016A
:104EA000455E5F4F698D7A8DCE0101960E946A271B
:104EB0004D815E8157FD0AC02F8138854217530707
:104EC0000CF49A01F801E20FF31F10822E96E4E031
:104ED0000C94672AABE0B0E0E0E7F7E20C943D2ADF
:104EE0006C017B018A01FC0117821682838181FF9C
:104EF000CCC1CE0101963C01F6019381F70193FDEF
:104F0000859193FF81917F01882309F4BAC185328D
:104F100039F493FD859193FF81917F01853229F4C6
:104F2000B60190E00E946129E7CF912C212C312C11
:104F3000FFE1F315D8F08B3279F038F4803279F054
:104F40008332A1F4232D20611DC08D3261F08033A6
:104F500069F4232D216016C0832D8260382EE32D45
:104F6000E4603E2E2AC0F32DF8601DC037FC2DC032
:104F700020ED280F2A3040F08E32B9F436FC81C182
:104F8000232D2064322E19C036FE06C08AE0989E7A
:104F9000200D1124922E11C0EAE02E9E200D112426
:104FA000222EF32DF0623F2E08C08C3621F4832D83
:104FB0008068382E02C0883641F4F70193FD859150
:104FC00093FF81917F018111B3CF982F9F7D9554DD
:104FD000933028F40C5F1F4F9FE399830DC08336F5
:104FE00031F0833771F0833509F059C021C0F801E1
:104FF000808189830E5F1F4F88248394912C5301F5
:1050000013C02801F2E04F0E511CF801A080B180BE
:1050100036FE03C0692D70E002C06FEF7FEFC5015F
:105020000E9456294C018201F32DFF773F2E16C0B6
:10503000280122E0420E511CF801A080B18036FE0A
:1050400003C0692D70E002C06FEF7FEFC5010E94C1
:105050004B294C01F32DF0683F2E820133FC1BC01D
:10506000822D90E088169906B0F4B60180E290E0B7
:105070000E9461292A94F4CFF50137FC859137FE0F
:1050800081915F01B60190E00E94612921102A946C
:1050900021E0821A91088114910471F7E8C08436E6
:1050A00011F0893641F5F80137FE07C06081718142
:1050B000828193810C5F1F4F08C060817181072E30
:1050C000000C880B990B0E5F1F4FF32DFF763F2EC0
:1050D00097FF09C090958095709561957F4F8F4F90
:1050E0009F4FF0683F2E2AE030E0A3010E949D29E7
:1050F000882E861845C0853731F4232D2F7EB22E99
:105100002AE030E025C0932D997FB92E8F36C1F06B
:1051100018F4883579F0B5C0803719F0883721F058
:10512000B0C0E92FE061BE2EB4FE0DC0FB2DF460CF
:10513000BF2E09C034FE0AC0292F2660B22E06C039
:1051400028E030E005C020E130E002C020E132E09C
:10515000F801B7FE07C060817181828193810C5F85
:105160001F4F06C06081718180E090E00E5F1F4F8D
:10517000A3010E949D29882E8618FB2DFF773F2EC4
:1051800036FE0DC0232D2E7FA22E891458F434FE36
:105190000BC032FC09C0832D8E7EA82E05C0B82C12
:1051A000A32C03C0B82C01C0B92CA4FE0FC0FE0173
:1051B000E80DF11D8081803321F49A2D997EA92E6E
:1051C00009C0A2FE06C0B394B39404C08A2D8678A9
:1051D00009F0B394A3FC11C0A0FE06C0B21488F479
:1051E000280C922C9B180EC0B21460F4B60180E219
:1051F00090E00E946129B394F7CFB21418F42B18F1
:1052000002C0982C212CA4FE10C0B60180E390E0CF
:105210000E946129A2FE17C0A1FC03C088E790E0AC
:1052200002C088E590E0B6010CC08A2D867859F05E
:10523000A1FE02C08BE201C080E2A7FC8DE2B601B4
:1052400090E00E946129891438F4B60180E390E06F
:105250000E9461299A94F7CF8A94F301E80DF11D19
:105260008081B60190E00E9461298110F5CF222053
:1052700009F442CEB60180E290E00E9461292A94AE
:10528000F6CFF6018681978102C08FEF9FEF2B96B4
:10529000E2E10C94592AFC01059061507040011024
:1052A000D8F7809590958E0F9F1F0895FC0161504F
:1052B000704001900110D8F7809590958E0F9F1F38
:1052C00008950F931F93CF93DF93FB01238121FD5B
:1052D00003C08FEF9FEF2CC022FF16C0468157817D
:1052E000248135814217530744F4A081B1819D0187
:1052F0002F5F3F4F318320838C93268137812F5F2F
:105300003F4F3783268314C08B01EC01FB010084DF
:10531000F185E02D0995892BE1F6D80116968D913E
:105320009C911797019617969C938E931697CE0192
:10533000DF91CF911F910F910895FA01AA2728308C
:1053400051F1203181F1E8946F936E7F6E5F7F4F52
:105350008F4F9F4FAF4FB1E03ED0B4E03CD0670FCE
:10536000781F891F9A1FA11D680F791F8A1F911D21
:10537000A11D6A0F711D811D911DA11D20D009F471
:1053800068943F912AE0269F11243019305D3193B3
:10539000DEF6CF010895462F4770405D4193B3E09C
:1053A0000FD0C9F7F6CF462F4F70405D4A3318F043
:1053B000495D31FD4052419302D0A9F7EACFB4E0F4
:1053C000A6959795879577956795BA95C9F70097AC
:1053D0006105710508959B01AC010A2E069457954D
:1053E000479537952795BA95C9F7620F731F841FA4
:1053F000951FA01D0895F999FECF92BD81BDF89A21
:10540000992780B50895A8E1B0E042E050E00C94FF
:105410002F2A262FF999FECF92BD81BDF89A0197C8
:1054200000B4021639F01FBA20BD0FB6F894FA9AEC
:10543000F99A0FBE08950396272F0E940A2A0E9408
:10544000092A252F0E940A2A242F0C940A2A019641
:10545000272F0E940A2A0C94092ADC01CB01FC01A7
:10546000F999FECF06C0F2BDE1BDF89A319600B4BD
:105470000D9241505040B8F708952F923F924F92AD
:105480005F926F927F928F929F92AF92BF92CF92D4
:10549000DF92EF92FF920F931F93CF93DF93CDB7DD
:1054A000DEB7CA1BDB0B0FB6F894DEBF0FBECDBF55
:1054B00009942A88398848885F846E847D848C8426
:1054C0009B84AA84B984C884DF80EE80FD800C812F
:1054D0001B81AA81B981CE0FD11D0FB6F894DEBF12
:0C54E0000FBECDBFED010895F894FFCF82
:1054EC0064001602280850011E0A140140FFC51F53
:1054FC00FC1FC91F73206120C81F01E200E900EAEC
:10550C0000B500B600B700CD008301CC008A019233
:10551C000194012102230224022502260227022AD9
:10552C0002B300B4006F007000818283E200E900D6
:10553C00EA00B500B600B700CD008301CC008A01AB
:10554C009201940121022302240225022602270241
:10555C002A02B300B4006F007000818283F5F6F765
:10556C00F0F1F4363597679637929390914C005240
:10557C00004D00300041542B424C45504F57455282
:0A558C004C4556454C3D25640000D7
:00000001FF
